:020000040800F2
:10000000185400202902000839250008D11E0008D4
:100010003525000821050008592C000800000000C3
:10002000000000000000000000000000E1250008C2
:10003000F1050008000000007125000845260008B1
:10004000430200084302000843020008430200087C
:10005000430200084302000843020008430200086C
:1000600043020008F50500080106000843020008E5
:100070004302000825050008430200084302000867
:10008000430200084302000843020008430200083C
:100090004302000843020008430200080D0600085E
:1000A000430200084302000843020008430200081C
:1000B000430200084302000843020008430200080C
:1000C00043020008430200084302000843020008FC
:1000D00043020008430200084302000843020008EC
:1000E00043020008430200084302000843020008DC
:1000F00043020008430200084302000843020008CC
:1001000043020008430200084302000843020008BB
:1001100043020008430200084302000843020008AB
:10012000430200083505000845050008550500088C
:10013000430200084302000843020008430200088B
:10014000430200084302000843020008430200087B
:10015000430200084302000843020008492C00083B
:10016000430200084302000843020008430200085B
:100170004302000843020008430200080000000098
:10018000430200084302000800F002F800F03CF8C7
:100190000AA090E8000C82448344AAF10107DA45E2
:1001A00001D100F031F8AFF2090EBAE80F0013F0F8
:1001B000010F18BFFB1A43F00103184768490000FC
:1001C00088490000103A24BF78C878C1FAD852078D
:1001D00024BF30C830C144BF04680C6070470000C1
:1001E0000023002400250026103A28BF78C1FBD840
:1001F000520728BF30C148BF0B6070471FB504F0DD
:100200005FFC1FBD10B510BD00F054F91146FFF79B
:10021000F5FF02F065FD00F072F903B4FFF7F2FF9D
:1002200003BC00F075F90000094880470948004701
:10023000FEE7FEE7FEE7FEE7FEE7FEE7FEE7FEE796
:10024000FEE7FEE704480549054A064B70470000F3
:10025000FD26000889010008184E002018540020CF
:10026000185000201850002053EA020C00F069805A
:100270002DE9F04B4FF00006002B1FBFB3FA83F5BA
:1002800003FA05F424FA05F65E4012BF1643B2FAEB
:1002900082F502FA05F4C5F120051EBF22FA05FC1D
:1002A00044EA0C04203556EA044C4FEA144418BFC3
:1002B000641C4FF000084FF00009904271EB030CF2
:1002C00039D3002919BFB1FA81F701FA07F6B0FA5C
:1002D00080F700FA07F6C7F120071EBF20FA07FCD7
:1002E00046EA0C062037B6FBF4FCA7EB0507103FE7
:1002F00007F01F0BCBF120062CFA06F60CFA0BFBCD
:1003000044BFB3460026202FA4BF5E464FF0000B2B
:100310005BEA060C08BF4FF0010B19EB0B0948EB29
:100320000608ABFB027C06FB02CC0BFB03CCC01B1C
:1003300071EB0C01C1E70B46024641464846BDE859
:10034000F08B13B5084318BF4FF0FF300146AFF3F1
:100350000080BDE81C407047032A40F2308010F056
:10036000030C00F0158011F8013BBCF1020F624450
:1003700098BF11F801CB00F8013B38BF11F8013BE1
:10038000A2F1040298BF00F801CB38BF00F8013B8E
:1003900011F0030300F05780083AC0F0088051F8CC
:1003A000043B083A51F804CBA0E80810F5E7121D09
:1003B0005CBF51F8043B40F8043BAFF30080D20728
:1003C00024BF11F8013B11F801CB48BF11F8012BF4
:1003D00024BF00F8013B00F801CB48BF00F8012B17
:1003E000704702F0FF0343EA032242EA024200F0B0
:1003F00002B84FF0000200B51346944696462039E5
:1004000022BFA0E80C50A0E80C50B1F12001BFF4CD
:10041000F7AF090728BFA0E80C5048BF0CC05DF833
:1004200004EB890028BF40F8042B08BF704748BF81
:1004300020F8022B11F0804F18BF00F8012B7047F5
:1004400070477047704710B5203AC0F00B80B1E894
:100450001850A0E81850B1E81850A0E81850203AF9
:10046000BFF4F5AF5FEA027C24BFB1E81850A0E802
:10047000185044BF18C918C0BDE810405FEA827C1C
:1004800024BF51F8043B40F8043B08BF7047D20733
:1004900028BF31F8023B48BF11F8012B28BF20F8D4
:1004A000023B48BF00F8012B70470000004870472E
:1004B000100000207546FFF7F9FFAE4605006946BB
:1004C000534620F00700854618B020B5FFF7BAFE66
:1004D000BDE820404FF000064FF000074FF0000845
:1004E0004FF0000BAC46ACE8C009ACE8C009ACE882
:1004F000C009ACE8C00921F007018D46704710B56E
:100500000446AFF300802046BDE81040FFF785BEEB
:1005100001491820ABBEFEE726000200704700002C
:10052000FEE7000080B540F2DC00C2F2000000F0FF
:10053000C9F880BD80B540F2FC10C2F2000000F0A6
:10054000C1F880BD80B540F23C10C2F2000000F05E
:10055000B9F880BD80B540F29C10C2F2000000F0F6
:10056000B1F880BDD0F800C06FF00F024AF6AB239F
:1005700052FA8CF2CAF6AA230146A2FB0330000904
:1005800005A31B5C40F2FF302CEA00005F2A88BF05
:100590000430C1E916037047000610160006101655
:1005A0008269816AB2F5005F06D06AB9022912D069
:1005B000012914D0D1B90EE0032917D8DFE801F0E2
:1005C000020B020F0120704703293CBF0120704736
:1005D0001CBF00207047C06AC0F300607047C06A4B
:1005E000A0F1C070B0FA80F0400970470020704759
:1005F0007047000080B5082000F0A8F980BD000019
:1006000080B5102000F0A2F980BD000080B5202048
:1006100000F09CF980BD000072B600BFFEE700004C
:1006200070B5866D044600F073FA94F8351002290F
:1006300025D105462068216C026822F0160202606E
:10064000426922F08002426109B9A16C19B10168C6
:1006500021F008010160016821F00101016000BF83
:1006600020680068C0070ED000F052FA401B062830
:10067000F6D320206065032084F835000CE080204C
:100680006065012008E0E06D3F2101FA00F0B060F4
:10069000012084F835000020002184F8341070BD5A
:1006A00090F83510022909D1052180F8351000682D
:1006B000016821F00101016000207047802141653F
:1006C00001207047F0B581B004460020009040F250
:1006D0000000C2F200000268D4E9166048F2B513C7
:1006E00037680821C1F64E3381403942A2FB032509
:1006F0000CD0226813685B0708D5136823F0040345
:100700001360B160616D41F00101616501218140BB
:10071000394208D022685269120604D5B160616D71
:1007200041F00201616504218140394208D022680C
:100730001268920704D5B160616D41F004016165F2
:1007400010218140394215D020680268120711D566
:10075000B16002680168520306D4C90506D4016875
:1007600021F00801016001E0080342D4216C09B1C5
:1007700020468847E16D202000FA01F23A4244D039
:1007800020680368DB0640D5B26094F83530026813
:10079000052B1ED122F016020260426922F080026F
:1007A0004261226C0AB9A26C1AB1026822F00802F6
:1007B00002603F208840B060012084F83500216D40
:1007C0000020002984F8340040D02046884701B03A
:1007D000F0BD0168520310D4C90512D4016821F09C
:1007E00010010160012084F83500002084F83400F5
:1007F00007E0A16C0029BBD1BCE7080301D4616C00
:1008000000E0E16B09B120468847606DF0B1606D92
:10081000C00717D0052084F835002068A90A0268AF
:1008200022F00102026000BF009A01328A42009267
:1008300002D80268D207F7D1012084F835000020E1
:1008400084F83400E16C09B12046884701B0F0BD5E
:100850002DE9F041044600F05BF9C4B105460220E1
:1008600084F835000020216884F83400086820F0FE
:100870000100086026683068C0070BD000F048F916
:10088000401B0528F6D903212022032042E0012045
:10089000BDE8F081306848F23F01CFF21001251D1C
:1008A00000EA010C2ECDD4E9050E41EA0C011143FA
:1008B00019432943D4E90778084340EA0E01606AE6
:1008C0003943042841EA080103D1D4E90B23114339
:1008D000194331607169042821F0070141EA0005DC
:1008E0000CD1D4E90A1045EA010538B12046FFF7DA
:1008F00057FE18B10121402201200BE0204675610E
:10090000FFF730FEE16D3F2202FA01F18160002223
:1009100001210020626584F83510BDE8F0810000F7
:1009200070B540F2700604460025C2F2000603E0EE
:100930000135102D08BF70BD24FA05F0C007F7D0AF
:1009400056F82500002818BF8047F1E780B543F628
:100950001441C4F201010A68024208BF80BD086068
:10096000FFF7DEFF80BD00002DE9F04F83B000F1FE
:100970003E4202F1FF724FEAB22241F60047019275
:10098000C4F2020708224FF0010E00254FF0000AC2
:100990004FF00008B84208BF072200920AE000BFEB
:1009A00008F101080AF1040AB8F1100F05F1020577
:1009B00000F0A4800C680EFA08FB14EA0B09EFD0D3
:1009C0004C6804F0030CACF1010EBEF1010F11D81C
:1009D0000322876802FA05F6CA68B743AA403A4379
:1009E00082604268C4F3001722EA0B0207FA08F794
:1009F0003A434260BCF1030F1CD0C26803238E68E7
:100A000003FA05F7BA4306FA05F73A43BCF1020FB9
:100A1000C2600FD16FF0030202EA580202440AF0EA
:100A20001C060F23176A03FA06F40B69A743B340A9
:100A30003B431362026803234F68AB409A4307F0BD
:100A40000303AB401A4317F4403F4FF0010E02601E
:100A5000A6D0002243F644030292C4F202031A68AD
:100A600043F6004442F480421A601A68C4F201045A
:100A700002F480420292029A28F003024FF6084BD9
:100A80002244CFF6FF7B52F80B300AF00C070F26FA
:100A9000BE4023EA060C019B009E072B38BF1E4672
:100AA00006FA07F747EA0C0342F80B30A2684B68D6
:100AB00042EA090743F60C4CDE0258BF22EA090756
:100AC000A760C4F2010CDCF800209E0242EA09078C
:100AD00058BF22EA0907CCF8007062689E0342EA18
:100AE000090758BF22EA090767602268DB0342EA68
:100AF000090358BF22EA0903236051E703B0BDE8A8
:100B0000F08F0000002A08BF0904816170470000CF
:100B100044F23860C2F2000000687047F0B581B05E
:100B2000B0B3044690F83D0028B9002084F83C009A
:100B3000204600F0BFF8242084F83D0020680168BA
:100B400021F001010160016841F400410160016888
:100B500021F40041016000F09DFA48F28041C0F2AA
:100B60001E0140F60012656888424FF00001C0F295
:100B70003D0248F2A16C4FF0000338BF01219042C2
:100B8000C0F2010C38BF0123654538BF0B4613B1D5
:100B9000012001B0F0BD4DF68361C4F21B31A0FB12
:100BA000011221684FEA924E4B684FF4967623F07B
:100BB0003F0343EA92434B6044F6D3530F6A0EFB64
:100BC00006F6C1F26203A6FB033627F03F03B7091E
:100BD000654538BF970C7A1C1A430A62CA6948F205
:100BE000A0674CF6FF73C0F20107BD4222EA030C76
:100BF0000AD801386A00B0FBF2F001306FF31F3001
:100C0000042898BF04202BE0A368A0F1010E9BB13B
:100C100019206843BEFBF0F00422013062F31F305C
:100C2000000512D09BB119206843BEFBF0F00422EE
:100C3000013062F31F3011E005EB4500BEFBF0F020
:100C400001306FF31F300005ECD1012008E005EB07
:100C50004500BEFBF0F001306FF31F3040F4004060
:100C600040EA0C00C8610868D4E9072320F0C000FE
:100C7000104318430860886848F2FF3204F10C07FB
:100C800090438CCF18431043A6698860C86820F051
:100C9000FF0038433043C860086840F00100086036
:100CA00000202021206484F83D10206384F83E0059
:100CB00001B0F0BD2DE9F04F87B00446006845F65D
:100CC0000041C4F2000100278842CDE90577CDE953
:100CD0000377029732D045F60001C4F20001884242
:100CE00040F09080002443F630050194C4F20205E0
:100CF0002868122140F020002860286800F02000B9
:100D00000190019803200290059004200690002095
:100D1000C4F20200CDE9031400F5A05002A9FFF7C8
:100D200023FE0194286940F480002861286900F4BA
:100D300080000190019807B0BDE8F08F43F63005C0
:100D40000197C4F20205286840F2000840F0040050
:100D500028602868C4F2020800F00400019001989D
:100D60000197286802AE40F00100286028684FF023
:100D7000120900F00100019001984FF400700290F8
:100D80004FF0030A4FF0040B08F500603146CDE93F
:100D90000397CDF814A0CDF818B0FFF7E5FD4FF498
:100DA0008070CDE9020904A880E8800C40463146F5
:100DB000FFF7DAFD019728694FF0C06140F40000A9
:100DC0002861286940F2DC0500F4000001900198D8
:100DD00046F24000C2F20005C4F202004FF4806205
:100DE00085E883002846C5E90372C5E90577C5E9AA
:100DF00007776F62FFF72CFD002818BFFFF70CFC88
:100E0000A563AC6307B0BDE8F08F000040F20400BA
:100E100044F23861C2F20000C2F2000100780A68B0
:100E2000104408607047000080B543F60040C4F2EB
:100E30000200016841F400710160016841F48061C1
:100E40000160016841F480710160032000F068F8DE
:100E50000F2000F005F800F02BF8002080BD000006
:100E6000B0B540F20402C2F2000240F20001127872
:100E7000C2F200014FF47A730968B3FBF2F2044640
:100E8000B1FBF2F1084600F0F3FB0F2C4FF0010527
:100E90000CD858B94FF0FF3021460022002500F051
:100EA0002FF840F20800C2F2000004602846B0BDEE
:100EB00080B582B0002043F640010190C4F20201E7
:100EC0004A6842F480424A604A6802F480420192D1
:100ED000019A00900868002240F08050086008687D
:100EE0000F2100F08050009000986FF0010000F09A
:100EF00007F802B080BD000080B501F0AFFE80BDF4
:100F000070B514460D46064601F0B8FE2946224645
:100F100001F014FB0146304601F0B8FE70BD000040
:100F200080B501F0CDFE80BD2DE9F041002800F034
:100F30008B8043F60808C4F202080446D8F8F80388
:100F40000D4600F00700884207D288F8F853D8F819
:100F5000F80300F00700A84276D12068810717D572
:100F6000410705D5D8F8001041F4E051C8F8001049
:100F7000010705D5D8F8001041F46041C8F8001009
:100F8000D8F80010A26821F0F0011143C8F8001051
:100F9000C0073FD1D8F8F80300F00700A84207D9EE
:100FA00088F8F853D8F8F80300F00700A8424BD1AE
:100FB0002068410707D5D8F80010E26821F4E05115
:100FC0001143C8F80010000708D5D8F800002169BF
:100FD00020F4604040EAC100C8F8000000F07EF84C
:100FE000D8F8001044F6DA22C1F30311C0F600026B
:100FF000515C40F2000220FA01F140F20800C2F216
:1010000000000068C2F200021160FFF729FF002013
:10101000BDE8F0816068811E022907D258F8081CDB
:1010200089015CBF0120BDE8F08110E0012807D1F3
:1010300058F8081C89035CBF0120BDE8F08106E078
:1010400058F8081C890702D40120BDE8F081D8F8BF
:10105000001021F003010843C8F80000FFF758FD15
:10106000064641F2883700BFD8F80000616800F0FA
:101070000C00B0EB810F8DD0FFF74AFD801BB8420A
:10108000F2D90320BDE8F08140F20000C2F2000076
:101090000068704780B5FFF7F7FF43F60801C4F218
:1010A0000201096844F6EA22C1F38221C0F6000277
:1010B000515CC84080BD000080B5FFF7E5FF43F6F6
:1010C0000801C4F20201096844F6EA22C1F3423180
:1010D000C0F60002515CC84080BD000010B543F668
:1010E0000404C4F20204606800F00C0008280AD06E
:1010F000042819BF42F20040C0F2F40041F600306B
:10110000C0F2B70010BD206821682368490241F68B
:101110000031C0F2B70100F03F02C3F388105CBF9A
:1011200042F20041C0F2F401A1FB00010023FFF7ED
:101130009BF821680222C1F3014102EB4101B0FB9F
:10114000F1F010BD2DE9F04182B0002800F0A2803E
:101150000446007843F60006C007C4F2020643D0F6
:10116000B06800F00C00042805D1306880033BD53E
:101170006068C8BB8EE0B06800F00C00082802D19F
:1011800070684002F1D46568B5F5A02F0AD0B5F5B6
:10119000803F0BD0306820F480303060306820F41D
:1011A000802006E0306840F480203060306840F4F1
:1011B00080303060FFF7ACFC002D054611D000BF39
:1011C0003068800310D4FFF7A3FC401B6428F7D9D4
:1011D00022E100BFFFF79CFC401B64284FF0030096
:1011E00055D830688003F5D4207880071AD5B068C8
:1011F00010F00C0F09D0B06800F00C00082840F087
:101200008A807068400200F186803068800702D5CD
:10121000E06801283ED13068216920F0F80040EAFA
:10122000C10030602078000738D4207840074CD4C3
:10123000A5695DB3B06800F00C00082840F09E80FE
:10124000012D27D07068E16900F480028A4221D123
:10125000216A00F03F028A421CD147F6C071626ADF
:101260000140B1EB821F15D1A26A0023CFF6FF73B4
:1012700003EBC23200F440316FF30F02914209D107
:10128000E16A00F07060B0EB016F03D1002002B0A2
:10129000BDE8F081012002B0BDE8F081606900285E
:1012A00040F20000C4F2472057D00121C0F8801E50
:1012B000FFF72EFC054600BF706F8007B5D4FFF71F
:1012C00027FC401B0228F7D9A6E0306C10F08058AC
:1012D0000AD100200190306C40F080503064306CB6
:1012E00000F080500190019847F20007C4F2000717
:1012F0003868C00524D4386840F480703860FFF73F
:1013000007FC05463868C0051AD4FFF701FC401BEE
:101310000228F7D980E0E068002851D00020C4F20C
:10132000472001210160FFF7F3FB05463068800785
:101330003FF571AFFFF7ECFB401B0228F6D96BE0DD
:10134000A568052D50D0012D52D0306F20F001003E
:101350003067306F20F004004DE00021C0F8801E9F
:10136000FFF7D6FB054600BF706F80077FF55DAFC6
:10137000FFF7CEFB401B0228F6D94DE00027C4F250
:10138000472700203866FFF7C3FB022D05460BD127
:101390003068800158D5FFF7BBFB401B02284FF097
:1013A0000300F5D973E700BF306880017FF56EAFA9
:1013B000FFF7AEFB401B02284FF00300F4D966E7AD
:1013C0000020C4F2472000210160FFF7A1FB054681
:1013D000306880077FF526AFFFF79AFB401B022895
:1013E0004FF00300F4D952E7306F40F0040030674B
:1013F000306F40F001003067FFF78AFB002D054693
:1014000041F2883714D000BF306F800713D4FFF744
:101410007FFB401BB842F7D9032002B0BDE8F08142
:10142000FFF776FB401BB8424FF003003FF62FAFAB
:10143000306F8007F4D4B8F1000F7FF4F9AE306C50
:1014400020F080503064F3E604F11C052FCD0843F2
:101450000021CFF6FF7140EA821001EBC3316FF338
:101460000F0140EA05600843706001203866FFF70D
:101470004FFB0446306880013FF508AFFFF748FB9B
:10148000001B02284FF00300F4D900E770B538B113
:101490000446406A30B10020206104F1140007E0E6
:1014A000012070BD6068B0F5827F03D004F11C009C
:1014B000002101600026A66294F8510020B9204660
:1014C00084F8506000F03CF8022084F8510094E861
:1014D0000F0001F48271056802F4044225F0400512
:1014E0000560114403F400622369114403F0020211
:1014F0006369114403F00102A369E569114403F42F
:101500000072114405F03802256A114405F080028A
:10151000A56A114305F4005211430160626A042177
:1015200001EA134102F0100211444160C16921F443
:101530000061C1610120666584F85100304670BDCC
:101540002DE9F04F87B0044643F200070068C4F26B
:1015500001070026B8420696CDE904660396029676
:1015600002D007B0BDE8F08F43F630000196C4F218
:101570000200416902AD41F48051416141694FF07F
:10158000020901F4805101910199019601684FF01F
:10159000010A41F00201016001684FF0030B01F004
:1015A000020101910199019601684FF0050841F08F
:1015B000010101600068294600F0010001900198D6
:1015C0001820029007F55440CDF80C90CDF810A0EB
:1015D000CDF814B0CDF81880FFF7C6F9802002A925
:1015E00081E8010ECDF8188046F2404807F55040DA
:1015F0002946C4F20208FFF7B7F940F23C15C2F2DF
:1016000000054FF0C0674FF480692846C5E90087A0
:10161000C5E90266C5E90496C5E90666C5E9086636
:10162000FFF716F9002818BFFEF7F6FFE564AC6374
:1016300040F29C1508F11800C2F200054021C5E9EE
:10164000000705F10800002280E806022846C5E9E7
:101650000522C5E907226A62FFF7FAF8002818BFD9
:10166000FEF7DAFFA564AC6307B0BDE8F08F0000B9
:1016700080B500F0CFFF80BDB0B590F83C20012AC6
:1016800004BF0220B0BD01F108053CCDD1E900CE78
:1016900023F47C5322F470521A432EF4F0431A437D
:1016A0002CF4E0431A4324F4C0431A432A43C96983
:1016B00022F48042036811435964002180F83C10F1
:1016C0000846B0BD10B590F83C20012A4FF0020248
:1016D00052D0012380F83C3080F83D200268D2F8D7
:1016E00004E0D2F808C00C682EF07003234341F2E6
:1016F000FF74C4F20004A24253600DDC40F2FF7399
:10170000C4F200039A4215DCB2F1804F29D040F2B6
:101710000043C4F2000322E040F2FF33C4F20103AD
:101720009A4212DC41F60003C4F200039A4218D038
:10173000002312E040F60003C4F200039A4210D0E6
:1017400040F60043C4F2000309E044F20003C4F28F
:1017500001039A4205D040F20043C4F201039A42C9
:1017600004D149682CF080031943916001210022C3
:1017700080F83D1080F83C20104610BD002804BFC2
:101780000120704710B5044690F83D0028B90020AC
:1017900084F83C00204600F01FF8022084F83D0049
:1017A0002068211D00F0B4FF012084F8460084F871
:1017B0003E0084F83F0084F8400084F8410084F83B
:1017C000420084F8430084F8440084F8450084F81B
:1017D0003D00002010BD000081B0006844F20041CF
:1017E000C4F20101884201D001B07047002000908E
:1017F00043F64400C4F20200016841F40031016084
:10180000006800F400300090009801B070470000BC
:1018100080B586B000684FF6FF71C4F200018842BF
:101820004FF000010591CDE90311CDE9011129DC4B
:1018300040F60001C4F2000188424AD040F600415F
:10184000C4F20001884240F082804FF0000C43F661
:101850003000CDF800C0C4F202000268002342F05C
:10186000800202600068022200F080000090009870
:101870004FF4E050019040F60040C4F2020000F541
:1018800080505CE044F20041C4F2010188423BD048
:101890000021C4F20101884259D14FF0000C43F6F7
:1018A0003000CDF800C0C4F20200026842F010021D
:1018B00002600068012200F01000009000984FF4D0
:1018C000D440019040F60040C4F2020000F5806070
:1018D00034E04FF0000C43F63000CDF800C0C4F205
:1018E00002000268002342F008020260006802223F
:1018F00000F00800009000984FF48040019040F6FE
:101900000040C4F202001AE00020009043F63000CC
:10191000C4F202000168032241F020010160006866
:101920004FF0020C00F02000009000984020019041
:1019300040F60040C4F2020000F5006002230221DC
:10194000CDE9021C01A9CDE90432FFF70DF806B07C
:1019500080BD0000B0B5044690F83C00012804BFEB
:101960000220B0BD0D464FEAB2010120032984F8E0
:101970003C0037D8DFE801F0020A1222206829462D
:1019800000F05CFF206850F8181F0EE02068294620
:1019900000F086FF206850F8181F16E020682946DE
:1019A00000F0B4FF206850F81C1F41F008010160EE
:1019B000016821F00401016029690FE020682946CF
:1019C00000F0D8FF206850F81C1F41F4006101604E
:1019D000016821F4806101602969090202681143EC
:1019E00001600020002184F83C10B0BD002804BF35
:1019F0000120704710B5044690F83D0028B900203A
:101A000084F83C00204600F01FF8022084F83D00D6
:101A10002068211D00F07CFE012084F8460084F837
:101A20003E0084F83F0084F8400084F8410084F8C8
:101A3000420084F8430084F8440084F8450084F8A8
:101A40003D00002010BD000083B0006840F600019A
:101A5000C4F2000188421BD040F60041C4F20001EC
:101A6000884226D00021C4F20101884230D10020F2
:101A7000029043F64000C4F20200416841F00101C7
:101A80004160406800F001000290029803B0704786
:101A90000020019043F64000C4F20200016841F0CA
:101AA00004010160006800F004000190019803B097
:101AB00070470020009043F64000C4F20200016825
:101AC00041F008010160006800F0080000900098F3
:101AD00003B070477047000080B500F0AFFF0228E8
:101AE00008BF80BD40F2B40100EBC000C2F20001AB
:101AF00001EB80000069002818BF804780BD00000E
:101B0000B0B582B0036804461868D9685A6900F015
:101B10002F05202D01F0200505D125B1204600F02C
:101B200097FF02B0B0BD5FEA007C1EBF02F0010E5D
:101B300001F4907212EB0E024AD1226B0840C106EA
:101B40003DD5012A3BD100200190186801905868CA
:101B5000019001985869400642D4A08DE18DE28D34
:101B6000002A1CBF401A5FEA004101D102B0B0BD9B
:101B7000216851E8031F226821F4907142E80313A1
:101B8000002BF5D1216851E8051F226821F00101E1
:101B900042E80513002BF5D1202184F842100021E2
:101BA000216300BF216851E8031F226821F0100162
:101BB00042E80313002BF5D10221616354E00106D2
:101BC00054D44006D2D5204600F02CFF02B0B0BD60
:101BD000C20718BF11F480725DD1420761D467E07B
:101BE000E06B016849688AB2002A44D0A38D9A420A
:101BF00041D2E185C069B0F5807F30D0206850E8DF
:101C0000030F216820F4807041E80302002AF5D117
:101C1000206850E8050F216820F0010041E8050226
:101C2000002AF5D1206850E8050F216820F0400017
:101C300041E80502002AF5D1202084F84200002066
:101C4000206300BF206850E8030F216820F01000D7
:101C500041E80302002AF5D1E06BFEF7E1FC022027
:101C60006063A08DE18D401A81B20FE0204600F044
:101C7000C1FF02B0B0BDA18D91427FF477AFC069C2
:101C8000B0F5807F7FF472AF022060632046FFF7DB
:101C900021FF02B0B0BD626C42F0010262644207F3
:101CA00006D5BEF1000F03D0626C42F002026264FE
:101CB000820706D5BEF1000F03D0626C42F0040229
:101CC0006264BCF1000F06D55EEA050203D0626CC7
:101CD00042F008026264626C002A3FF447AF084099
:101CE000800602D5204600F0B3FE20684069616C92
:101CF00000F0400001F00801401827D0204600F015
:101D000069FE2068406940061BD500BF206850E886
:101D1000050F216820F0400041E80502002AF5D1B6
:101D2000E06B70B142F6C511C0F600010165FEF727
:101D3000B7FC00283FF41AAFE06B016D884702B092
:101D4000B0BD2046FFF7C8FE02B0B0BD2046FFF789
:101D5000C3FE0020606402B0B0BD0000002804BFD4
:101D60000120704710B5044690F8410028B90020C2
:101D700084F84000204600F021F8242084F8410037
:101D80002068C16821F40051C160204600F0C4FE03
:101D90002068016921F490410161416921F02A0123
:101DA0004161C16841F40051C1600020202160649C
:101DB00084F8411084F84210606310BD70B586B09D
:101DC000044641F200402168C4F20100002681422D
:101DD0000596CDE903660296019601D006B070BD66
:101DE00043F630010096C4F202014A6900F58230E0
:101DF00042F020024A614A6902F020020092009AF1
:101E000000960A6842F040020A60096801F0400149
:101E1000009100994FF4844101910221CDE902160D
:101E2000032104910821059101A9FEF79DFD40F2CF
:101E3000FC1546F22840C2F20005C4F202004FF041
:101E400020614FF4806285E843002846C5E90362BB
:101E5000C5E90566C5E907666E62FEF7F9FC00286C
:101E600018BFFEF7D9FB472005210022E563AC63CC
:101E7000FFF746F84720FFF73FF806B070BD0000B7
:101E800080B500F0DBFD022808BF80BD40F2B40140
:101E900000EBC000C2F2000101EB8000C068002826
:101EA00018BF804780BD000080B500F0C7FD022844
:101EB00008BF80BD40F2B40100EBC000C2F20001D7
:101EC00001EB80004068002818BF804780BD0000FB
:101ED000FEE7000080B582B0002043F6300101909B
:101EE000C4F202010A6842F400120A600A6802F4AD
:101EF00000120192019A00900868002240F48000CC
:101F000008600868052100F48000009000980D200A
:101F1000FEF7F6FF0D20FEF7EFFF39200521002226
:101F2000FEF7EEFF3920FEF7E7FF3A2000210022FE
:101F3000FEF7E6FF3A20FEF7DFFF3B2005210022F7
:101F4000FEF7DEFF3B20FEF7D7FF02B080BD0000AA
:101F500080B542F20D6044F6F422C0F60000C0F6EF
:101F60000002002100F01AFF40F2D801C2F2000185
:101F7000086080BD2DE9F04F87B04FF0000943F6AF
:101F80003000CDF81890CDE90499CDE90299CDF84B
:101F90000490C4F20200016840F2004841F04001A0
:101FA00001600168C4F2020801F040010191019949
:101FB000CDF80490016808F5A05741F002010160D6
:101FC0000168002201F0020101910199CDF804900D
:101FD0000168402541F001010160016801F0010143
:101FE00001910199CDF80490016841F02001016050
:101FF000016801F0200101910199CDF80490016878
:1020000041F004010160016801F0040101910199AE
:10201000CDF80490016841F080010160016801F091
:10202000800101910199CDF80490016841F0080107
:102030000160016801F0080101910199CDF8049057
:10204000016841F0100101600068402100F01000BB
:10205000019001983846FEF755FDA8F58066304698
:10206000102101224FF0100A0124FEF74BFD4046DB
:102070004BF201010122FEF745FDCDE9025402AD0C
:1020800038462946CDE90444FEF76EFC082002904C
:102090004FF4041B38462946CDE903B4FEF764FC2F
:1020A00030462946CDE902A4CDE90444FEF75CFCA4
:1020B0003020CDE9020B08F5806029460494FEF734
:1020C00053FC4FF4304002A981E811020220059030
:1020D00040462946FEF748FC40462946CDE90244E1
:1020E000CDE90444FEF740FC4FF48040CDE90209FD
:1020F000404629460494FEF737FC092005210022BA
:10210000FEF7FEFE0920FEF7F7FE0A200521002259
:10211000FEF7F6FE0A20FEF7EFFE1720052100224B
:10212000FEF7EEFE1720FEF7E7FE07B0BDE8F08FE2
:1021300080B540F25C2045F60001C2F20000C4F216
:10214000000148F2A06200234FF4804CC0F201026B
:1021500080E80E00C0E9033CC0E90533C0E907335D
:10216000FEF7DCFC002818BFFEF756FA80BD000021
:1021700080B540F2B02045F60041C2F20000C4F242
:10218000000141F6802200234FF4804CC0F2060289
:1021900080E80E00C0E9033CC0E90533C0E907331D
:1021A000FEF7BCFC002818BFFEF736FA80BD000021
:1021B000B0B540F2043043F20001C2F20000C4F2B4
:1021C00001014FF48272002380E80E0000F10C013F
:1021D0004FF0020C4FF0010E4FF40074182581E807
:1021E00008500A21C0E90645C0E90833C0E90A31B0
:1021F000FFF74CF9002818BFFEF70EFAB0BD00003B
:1022000080B588B040F2A43044F200420021C2F20E
:102210000000C4F201024FF6FF730791CDE90511EA
:10222000CDE90311CDE90111C0E90021C0E9021394
:1022300001618161FFF7A2FA002818BFFEF7ECF9EF
:1022400040F2A430C2F20000FFF7D0FB002818BF14
:10225000FEF7E2F9602001900020CDE90200059030
:1022600040F2A430C2F2000001A90022FFF772FB85
:10227000002818BFFEF7D0F940F2A430C2F20000E7
:10228000FFF7C6FA08B080BD10B592B040F25C30DE
:1022900000210024C2F20000C4F201014FF6FF73D6
:1022A0001194CDE90F44CDE90D44CDE90B44CDE9BE
:1022B0000944CDE90744CDE90544CDE90344CDE91E
:1022C0000144A72280E81600C0E90334C0E90544B0
:1022D000FFF78CFB002818BFFEF79EF940F25C3038
:1022E000C2F2000010A9CDE91044FFF7EBF9002875
:1022F00018BFFEF791F9602009900020CDE90A008F
:10230000CDE90C00CDE90E0040F25C30C2F20000D5
:1023100009A90022FFF71EFB002818BFFEF77CF971
:1023200040F25C30C2F2000009A90422FFF712FB60
:10233000002818BFFEF770F940F25C30C2F20000CE
:1023400009A90822FFF706FB002818BFFEF764F969
:1023500040F25C30C2F2000009A90C22FFF7FAFA41
:10236000002818BFFEF758F900200590CDE90300BA
:10237000CDE901004FF40051089040F25C30069125
:10238000C2F2000001A9FFF777F9002818BFFEF795
:1023900043F940F25C30C2F20000FFF739FA12B0A4
:1023A00010BD000010B58AB040F2EC3040F60001DC
:1023B0000024C2F20000C4F200014FF6FF7309943A
:1023C000CDE90744CDE90544CDE90344CDE9014415
:1023D000A72280E81600C0E903348461FFF706FBFA
:1023E000002818BFFEF718F940F2EC30C2F20000E6
:1023F00008A9CDE90844FFF765F9002818BFFEF7E2
:102400000BF9602001900020CDE90200059040F218
:10241000EC30C2F2000001A90822FFF79BFA002865
:1024200018BFFEF7F9F840F2EC30C2F20000FFF7F7
:10243000EFF90AB010BD000010B58AB040F2344088
:1024400040F600410024C2F20000C4F200014FF047
:10245000FF330994CDE90744CDE90544CDE90344B0
:10246000CDE90144A72280E81600C0E90334846165
:10247000FFF7BCFA002818BFFEF7CEF840F2344050
:10248000C2F2000008A9CDE90844FFF71BF90028B3
:1024900018BFFEF7C1F8602001900020CDE90200CE
:1024A000059040F23440C2F2000001A90022FFF77B
:1024B00051FA002818BFFEF7AFF840F23440C2F2DC
:1024C000000001A90422FFF745FA002818BFFEF713
:1024D000A3F840F23440C2F2000001A90822FFF73D
:1024E00039FA002818BFFEF797F840F23440C2F2DC
:1024F0000000FFF78DF90AB010BD000080B540F272
:102500007C4041F20041C2F20000C4F2010100230C
:102510004FF00C0C4FF4E13280E80E00C0E90333B9
:10252000C0E905C3C361FFF719FC002818BFFEF717
:1025300073F880BDFEE70000FEE7000000F0070032
:1025400080F00703042B28BF04234FF0FF3C03381F
:102550000CFA03F338BF0020994381400CFA00F0D5
:1025600022EA00000843704700000000000000005D
:10257000EFF30980BFF36F8F154B1A681EF0100F31
:1025800008BF20ED108A20E9F04F10602DE9090006
:102590004FF0500080F31188BFF34F8FBFF36F8F60
:1025A00001F014FC4FF0000080F31188BDE8090031
:1025B00019680868B0E8F04F1EF0100F08BFB0ECC3
:1025C000108A80F30988BFF36F8F704700BF00BF88
:1025D000B80500200000000000000000000000001E
:1025E000074B19680868B0E8F04F80F30988BFF31B
:1025F0006F8F4FF0000080F31188704700BF00BF5D
:10260000B805002080B500F053FB80BD012000F02C
:1026100087FBFBE7B0B501380024B4EB106F1CBF9B
:102620000120B0BD4EF21005CEF2000568604FF0FB
:10263000FF300F2100F02AFB0720AC602860204605
:10264000B0BD000080B5FEF7E1FB01F0EBFF012813
:1026500018BF01F093FC80BD70B592B006AC204667
:102660003021FDF7C6FE002543F640000595CDE973
:102670000355CDE901550095C4F202000168022618
:1026800041F080510160006800F080500090009897
:1026900047F200000095C4F20000016841F4804157
:1026A0000160006800F480400090009801200690CE
:1026B0004FF4803007904FF480000D9006200E906C
:1026C000A820CDE90F060420119020460C96FEF7B5
:1026D00039FD88B90F20CDE901064FF4A0500490D0
:1026E0004FF48050059001A805210395FEF71CFCCE
:1026F000002804BF12B070BDFDF78EFF4EF6885063
:10270000CEF20000016841F47001016070470000E2
:10271000B0B540F6FF3E0568C4F2000E40F2004C32
:102720007045C4F2010C0FDCB0F1804F19D040F2BB
:102730000043C4F20003984213D040F60003C4F2F1
:10274000000398420DD011E040F60043C4F20003AC
:10275000984206D0604504D00023C4F20103984299
:1027600004D14B6825F0700243EA020541F6FF737D
:10277000C4F2000398420DDC70451FDCB0F1804FBD
:1027800041D040F20043C4F2000398423BD040F6EF
:10279000000321E043F6FF73C4F20103984220DCFA
:1027A00042F20003C4F2000398422CD00023C4F28A
:1027B0000103984227D0604525D029E040F6004328
:1027C000C4F2000398421ED041F60003C4F2000395
:1027D000984218D041F60043C4F20003984212D048
:1027E00016E044F20003C4F2010398420BD044F611
:1027F0000003C4F20103984205D044F20043C4F23E
:102800000103984204D1CB6825F4407243EA0205E3
:102810000A688C684B69C46240F4806482626445D3
:1028200004BF09690163026825F0800142F00402D7
:1028300019430260012242610160B0BDB0B5026A75
:10284000036A40F2004523F001030362D0F804E07C
:10285000D0F818C08C6822F0020240F48063C4F201
:102860000105AB4242EA040205D1CC6822F00C0219
:1028700024F0040422430C68AB4207D1D1E905538C
:102880002EF4407E45EA0E0545EA030E2CF0730354
:102890002343C0F804E08361496841630262B0BD2C
:1028A00070B5026A036A40F2004423F01003036229
:1028B000D0F804E0D0F818C08D6822F0200240F46F
:1028C0008063C4F20104A34242EA051207D1CD6835
:1028D0006FF0400622F0C00206EA05152A430D6893
:1028E000A34207D1D1E905642EF4406343EA86038D
:1028F00043EA840E2CF4E64343EA0523C0F804E0DF
:10290000836149688163026270BD000070B5026A2C
:10291000036A40F2004423F480730362D0F804E0B9
:10292000D0F81CC08D6822F4007240F48063C4F2B9
:102930000104A34242EA052207D1CD6840F2FF46D6
:102940002D0222F44062B5432A430D68A34207D109
:10295000D1E905642EF4405343EA061343EA041E0A
:102960002CF073032B43C0F804E0C3614968C163D2
:10297000026270BD70B5D0F820C0026A40F2004615
:1029800022F4805202624268C3690C68D1F808E000
:1029900040F48065C4F20106B54204D14D6922F4C9
:1029A000804242EA851223F4E64343EA042342606C
:1029B000C3612CF40056496846EA0E320164026293
:1029C00070BD000080B5806B0021C185FFF784F8E1
:1029D00080BD0000016851E8031F026821F4907176
:1029E00042E80313002BF5D1016851E8051F026886
:1029F00021F0010142E80513002BF5D1016B0129FB
:102A00000AD100BF016851E8031F026821F01001DC
:102A100042E80313002BF5D1202180F84210002159
:102A20000163704780B50168CA6822F04002CA603D
:102A3000202180F84110FFF737FA80BD006841F28D
:102A40000041C4F20101401A18BF01204000704744
:102A500080B582B090F8421022291ED18268B2F56A
:102A6000805F02D1016900294AD0816AB2F5805F96
:102A700007D00AB9026922B10268526802F07F02E7
:102A800001E0026852680A700121826A1144816281
:102A9000C18D01390A04C18501D002B080BD016831
:102AA000CA6822F02002CA60CA6822F48072CA6032
:102AB0004A6922F001024A61202180F84210002177
:102AC0004163026B012A23D1016300BF016851E811
:102AD000031F026821F0100142E80313002BF5D117
:102AE00001680A68D20606D5002201920A6801929E
:102AF000496801910199818DFEF7ECFF02B080BD1C
:102B00000168826A49686FF35F2111800221BCE786
:102B1000FFF7B6F902B080BD10B504460068D4E9ED
:102B200002C22369016921F44051114301616269C4
:102B300043EA0C01E3691143C268194349F20C638B
:102B40009A431143C1604169A26921F4407141F285
:102B50000043114340F48062C4F201039A42416190
:102B600002D1FEF7A9FA01E0FEF794FAE169636881
:102B70001922B1F5004FA0FB02011CD15A00DB0F56
:102B8000FDF772FB48F21F51C5F2EB11A0FB0123C8
:102B90005A096FF0630302FB0300322303EBC0000A
:102BA000A0FB01014FF4F87000EA111000EB0210D5
:102BB000C1F342111AE09A009B0FFDF755FB48F252
:102BC0001F51C5F2EB11A0FB01235A096FF06303FB
:102BD00002FB0300322303EB0010A0FB0101F020F5
:102BE00000EA511000EB0210C1F3431122680843C0
:102BF000906010BD90F84110212923D18168B1F572
:102C0000805F01D1016931B1016A02684B1C036226
:102C10000978516007E0016A036831F8022B6FF30D
:102C20005F225A600162C18C01390A04C18418BF55
:102C300070470068C16821F08001C160C16841F03F
:102C40004001C1607047000080B540F27C40C2F294
:102C50000000FEF755FF80BDFEE70000002848BFDA
:102C6000704700F01F01012202FA01F14EF200123A
:102C70004009CEF2000242F8201070474EF60C5088
:102C8000CEF200000068C0F3022070474EF61453E5
:102C900000F00F02CEF2000309011A4400F1604374
:102CA000B0F1FF3FC8BF03F56442117070470000E8
:102CB0004EF61F50CEF20000002101707047000058
:102CC0004EF60C51CEF200010A684FF6FF031A408F
:102CD00060F30A2242F0806040F0FD7008607047A7
:102CE000FEF7A2F8FFF7B8FCFFF744F9FFF7F2F898
:102CF000FFF71EFAFFF73CFAFFF7C6FAFFF752FBA1
:102D0000FFF79AFBFFF77CFAFFF752FAFFF7F6FBA3
:102D100000F016F8FFF71CF900F026F8FEE70000B7
:102D2000EFF3058100291CBF6FF0050070470028F4
:102D300004BF0020704780B500F074FF002080BD04
:102D4000EFF3058000281CBF6FF00500704740F2CC
:102D5000B000C2F200000168002911BF4FF0FF303F
:102D6000012101600020704710B5EFF305800028B5
:102D70001CBF6FF0050010BD40F2B004C2F20004A9
:102D8000206801281CBF4FF0FF3010BDFFF73AFC50
:102D90000220206000F0C0FF002010BD70B584B09C
:102DA0008E46002100280391EFF3058146D00029CB
:102DB00044D1FAB19369002B08BF1823382B16D8D9
:102DC0001179C90713D15569946811684FEA950CB8
:102DD000002D08BF4FF0800CFCB1D6685C2E1BD3D1
:102DE000D5B11569C5B10024012555B91BE00020F6
:102DF00004B070BD0124002118234FF0800C002581
:102E00008DB1946812690294CDE90032624673462E
:102E100001F0CCFB039011E00CB9D4689CB1002503
:102E20000024002DEDD14CB103AC00931FFA8CF2BD
:102E30007346019401F086FB012802D1039804B087
:102E400070BD0020E6E71469B4FA84F46409D6E79B
:102E5000F0B581B00D4644F6046140F2B856C2F2B6
:102E60000001C2F200060F6831680446081D00F038
:102E700061FD601C0AD14DB13068011D44F6DC5083
:102E8000C2F2000000F0B2FD01B0F0BD3068E419FC
:102E900044600AD340F2C850C2F2000000683168B2
:102EA000043100F085FD01B0F0BD40F2C050C2F227
:102EB000000000683168043100F07AFD44F6685083
:102EC000C2F2000001688C4238BF046001B0F0BD5E
:102ED00070B5044600F0A2FD44F23C60C2F200006E
:102EE000016840F2B85501310160C2F2000529685D
:102EF00044F6D056C2F2000641B1306860B9286885
:102F0000E16AC06A884298BF2C6005E02C600068C6
:102F1000012801D100F0C4F944F24860C2F2000077
:102F2000016801310160616444F24C61C2F2000148
:102F3000E06A0A68904288BF086040F2D05100EB16
:102F40008000C2F2000101EB8000211D00F04EFD67
:102F500000F088FD306880B12868E16AC06A884264
:102F600028BF70BD4EF60450CEF200004FF08051E5
:102F70000160BFF34F8FBFF36F8F70BD70B582B02C
:102F800000F04CFD44F60866C2F20006306850BB03
:102F900044F60854C2F20004204600F0F9FC44F65E
:102FA0001C55C2F20005284600F0F2FC40F2BC506D
:102FB000C2F20000046040F2CC50C2F2000040F2C5
:102FC000C44240F2645305600025C2F20002C2F21E
:102FD00000030A201021009500F0E8FF306010B1D6
:102FE00003A100F0E9FD00F03DFD02B070BD00BF9F
:102FF000546D725100000000F0B581B044F240659C
:10300000C2F200052868E0B144F6F05644F23C678D
:10301000C2F20006C2F2000700F000FDF068C468CA
:10302000201D00F087FC38680138386028680138B6
:10303000286000F017FD204600F058F828680028A6
:10304000EAD101B0F0BD000080B5026C002A08BFD3
:1030500080BDD0E902C31344C360634524BF036845
:10306000C360C36808461946FDF776F980BD0000C5
:1030700070B5866B036C0446E3B115461AB3E0687D
:103080001A46FDF769F9E168206C2268091A914235
:10309000E16003D2A16840420844E060A81EB0FA93
:1030A00080F040093146002E18BF01210840361A31
:1030B000002516E02068002598B9A06801F076FB8D
:1030C000A56005460DE060681A46FDF745F9216CDC
:1030D000D4E90102002508446060904224BF2068C2
:1030E0006060711C2846A16370BD000010B50446E5
:1030F00090F85900022808BF10BD012803D030B94C
:10310000206B00F0C7FC204600F0C4FC10BD4FF05F
:10311000500080F31188BFF36F8FBFF34F8F00BF54
:10312000FEE7000040F2BC51C2F2000109680A68E3
:10313000B2FA82F35B090360002A0EBF0020C86860
:103140000068704740F63020C2F20000C21D22F035
:10315000070210F0070CA0EB020318BF104644F65C
:10316000D452C2F200020021C2E900014FF47052B1
:10317000BCF1000F18BF03F570520244083A40F248
:10318000C45322F00702C2F200031A60C2E9001120
:10319000111A1A68C0E9002144F66450C2F2000016
:1031A000016044F65C50C2F20000016044F6305009
:1031B000C2F20000012101707047000040F2D054BB
:1031C0004EF60455C2F20004CEF200054FF08056D0
:1031D000FFF712FF20680228FAD32E60BFF34F8F4B
:1031E000BFF36F8FF4E70000B0B5049D002914BF52
:1031F0002A602D60C5E90F01284601211C4600F018
:1032000021FF85F84C40B0BD2DE9F0470A9C82466D
:10321000206B16460F46DDE908599100A522984615
:10322000FDF7DFF8206B00EB8600A0F1040020F032
:1032300007067FB104F13400002100BF7A5C4254DC
:103240007A5C1AB10F2901F10101F7D3002084F84B
:10325000430002E0002084F834000027201D372DB1
:1032600028BF3725E562C4E9135700F09DFB04F140
:10327000180000F099FBC5F13800A06130465146B6
:10328000424624616462676584F8587000F03EFB32
:10329000B9F1000F206018BFC9F80040BDE8F08701
:1032A000B0B540F2D0550024C2F20005281900F054
:1032B0006FFB1434B4F58C6FF8D144F63454C2F279
:1032C0000004204600F064FB44F64855C2F20005B5
:1032D000284600F05DFB44F67C50C2F2000000F08E
:1032E00057FB44F6F050C2F2000000F051FB44F6E8
:1032F000DC50C2F2000000F04BFB40F2C050C2F2C2
:103300000000046040F2C850C2F200000560B0BD89
:1033100080B544F6D452C2F2000200BF11461268D2
:103320008242FBD3D1F804C001EB0C03834203D1EA
:103330004068604448600846D0F804C000EB0C03C5
:10334000934201D013460BE040F2C453C2F2000393
:103350001B689A4204D0D2E9003E0EEB0C02426098
:103360008142036018BF086080BD000080B58C46B4
:10337000014641F804CF9445006108D99A4201D230
:103380009C4511D240F2BC50C2F2000007E08069B7
:10339000D21A824208D240F2CC50C2F20000006839
:1033A00000F006FB002080BD012080BD10B5044662
:1033B00000F034FBA06BB0FA80F0440900F052FB3F
:1033C000204610BD10B5044600F028FBA06BE16B51
:1033D000401AB0FA80F0440900F044FB204610BDCA
:1033E00008480068006880F308884FF0000080F308
:1033F000148862B661B6BFF34F8FBFF36F8F00DFE3
:1034000000BF00BF08ED00E070B582B040F2BC52D2
:10341000C2F2000212680546D2680E46D468201D2A
:1034200000F088FA94F82800410704D400F0FE0068
:1034300084F8280010E0A0693246411920462B4646
:10344000FFF794FF40B10026204600212A460023C2
:10345000009601F001FB20B1216A2046884702B0A6
:1034600070BD4FF0500080F31188BFF36F8FBFF332
:103470004F8F00BFFEE700002DE9F04186B044F613
:103480000867C2F20007386802A900224FF000085E
:1034900000F052FF00286AD001AC02AD0BE000F052
:1034A000FE0086F8280000BF38682946002200F098
:1034B00043FF00285BD00298B0F1FF3F03DCDDE959
:1034C00003200599904702980028EDD4049E706966
:1034D00010B1301D00F02EFA204600F0B3F802992A
:1034E0000929E1D80246DFE801F0080808052A3971
:1034F0000808052A96F82800D1E796F82800039BCB
:10350000B16940F0010086F8280019443046FFF701
:103510002DFF0028C8D0316A3046884796F8280029
:103520004007C1D50398B16900230A18304600212D
:10353000CDF8008001F090FA0028B5D123E096F88C
:10354000280040F00101039886F82810B06188B186
:10355000811830461346FFF709FFA5E796F82800C3
:1035600081073FF59CAF304600F094FA9CE706B027
:10357000BDE8F0814FF0500080F31188BFF36F8FEA
:10358000BFF34F8FFEE74FF0500080F31188BFF379
:103590006F8FBFF34F8F00BFFEE7000070B582B0A2
:1035A0000E46044600F00AFC01A800F04BF8019911
:1035B00019B101F08DF902B070BD05464EB9A542B2
:1035C00007D301F085F920462946FFF71DFF02B019
:1035D00070BD4EB140F2CC50C2F2000000680068ED
:1035E000B0FA80F0420900E0002244F60860C2F21E
:1035F00000000068611B00F0F3FA01F069F900288F
:10360000D9D14EF60450CEF200004FF08051016047
:10361000BFF34F8FBFF36F8F02B070BD40F2C05049
:10362000C2F200000168096821B10068C068C06882
:10363000406801E04FF0FF3044F66851C2F20001EB
:103640000860704770B5044601F000F840F2B456C7
:10365000C2F2000631680546884203D200F008F83D
:10366000012000E0002020602846356070BD000089
:103670002DE9F04182B040F2BC57C2F20007386831
:10368000016891B34FF0000809E000BF606038683E
:103690002946246100F08CF93868016829B3C068B4
:1036A000C4680668251D284600F044F9216A2046B2
:1036B000884794F828004007EED5A0693044B0420E
:1036C000E4D82046002132460023CDF8008001F0E6
:1036D000C3F90028E0D14FF0500080F31188BFF308
:1036E0006F8FBFF34F8F00BFFEE740F2CC51C2F2A5
:1036F00000010A6808603A6002B0BDE8F08100008D
:1037000081B00020009040F20C00C2F2000000687E
:103710004FF0500181F31188BFF36F8FBFF34F8FCC
:10372000013001D0FEE700BF00980028FCD001B0B6
:103730007047000082B001AC2046FFF7F3FC01990E
:10374000FFF72CFFFFF798FEF6E70000F0B581B019
:10375000044600F063F994F94560012E0FDB04F193
:10376000240500BF286850B1284601F069F80028F8
:1037700018BF00F08FFA70B2013E0128F2DCFF267C
:1037800084F8456000F06EF900F048F994F944704F
:10379000012F0EDB04F11005286850B1284601F016
:1037A0004FF8002818BF00F075FA78B2013F0128E1
:1037B000F2DC84F8446000F055F901B0F0BD00007F
:1037C0002DE9F04381B0044600F0F8FA40F2C45607
:1037D000C2F200063068002808BFFFF7B3FC44F6C9
:1037E0003058C2F2000898F80000002818BF4FF0C7
:1037F000004020420DD0002401F06AF860071ED07E
:103800004FF0500080F31188BFF36F8FBFF34F8FDD
:10381000FEE7C4B114F0070004F108011EBF081A46
:1038200000F108015FEA41700ED04FF0500080F3C4
:103830001188BFF36F8FBFF34F8F00BFFEE72046A5
:1038400001B0BDE8F083002144F65C59C2F20009E2
:10385000D9F800004A1E8242CDD244F6D450C2F2BA
:10386000000005682F4657F8042F8A4211D22B68B2
:103870005BB100BF1F4657F8042F28461D468A42F9
:1038800007D22B68002BF5D103E044F6D450C2F2E6
:10389000000033689D42AED004682B68521A112A8A
:1038A000036010D36818430709D04FF0500080F32D
:1038B0001188BFF36F8FBFF34F8F00BFFEE74260E9
:1038C0003960FFF725FD44F664503968D9F80020C7
:1038D000C2F200000368511A9942C9F8001038BFBB
:1038E000016098F80000396800284FF0000018BF08
:1038F00041F00041286044F67050C2F200000268B6
:1039000008343960511C016076E70000034643F239
:103910000170C0F600004FF0807C21F0010103E946
:1039200003106FF0020043F8240CA3F1440043F8A5
:10393000202C7047D0E9013201699A60D1F804C0A7
:1039400082688445536008BF4A60002202610868AB
:10395000013808600868704744F65003C2F200035B
:10396000036044F25060C2F20000086080201060E2
:103970007047000044F6AC43C2F20003036044F613
:10398000AC00C2F2000008604FF480701060704715
:103990004FF0FF31024642F8081F00214260C0E9A3
:1039A00003220160704700000021016170470000A0
:1039B00080B5D1F800C01CF1010207D000F1080366
:1039C0009E465B681A686245FAD901E0D0F810E0BB
:1039D000DEF8042008614A609160C1F808E0CEF882
:1039E000041001680131016080BD0000D0F800C002
:1039F000436808619A684B608A609A689960516070
:103A00000CF1010101607047DFF80C00016841F41E
:103A100070010160704700BF88ED00E04FF050007A
:103A200080F31188BFF36F8FBFF34F8F40F20C000C
:103A3000C2F2000001684A1C026001B170474EF6F4
:103A40000450CEF200000068000608BF70474FF037
:103A5000500080F31188BFF36F8FBFF34F8F00BF0B
:103A6000FEE7000040F20C00C2F20000016839B12C
:103A70000139016018BF7047002080F3118870473A
:103A80004FF0500080F31188BFF36F8FBFF34F8F5B
:103A9000FEE70000B0B5002808BFB0BD044644F6FC
:103AA0003050C2F20000007854F8041C002818BFFF
:103AB0004FF0004008420CD0A4F108052A6892B1EA
:103AC0004FF0500080F31188BFF36F8FBFF34F8F1B
:103AD000FEE74FF0500080F31188BFF36F8FBFF304
:103AE0004F8F00BFFEE721EA000044F8040C00F00D
:103AF00065F944F65C51C2F2000154F8040C0A68FE
:103B0000104408602846FFF703FC44F67450C2F2E4
:103B1000000001680131016000F0DAFEB0BD000074
:103B20004EF21000CEF2000000210160816040F2F0
:103B30000001C2F20001096844F6D352C1F26202E8
:103B4000A1FB02124FF0FF3101EB921141600721FE
:103B500001607047EFF30580102814D34EF2F03166
:103B6000CEF20001405C44F23061C2F200010978FB
:103B7000884208D24FF0500080F31188BFF36F8F56
:103B8000BFF34F8FFEE74EF60C50CEF2000044F22A
:103B900034610068C2F20001096800F4E060884204
:103BA00098BF70474FF0500080F31188BFF36F8FBC
:103BB000BFF34F8FFEE7000044F6905C0022C2F294
:103BC000000C00BF5CF8323023B10132082A08BF74
:103BD0007047F7E70CEBC2034CF83210586070479F
:103BE00070B515460E460446FFF718FF94F84400DA
:103BF000FF2804BF002084F8440094F84500FF2803
:103C000004BF002084F84500FFF72CFFA06B28B903
:103C100004F1240031462A4600F05EF82046FFF702
:103C200095FD70BD10B5D8B1044644F24460C2F2AF
:103C30000000006848B14FF0500080F31188BFF3D6
:103C40006F8FBFF34F8F00BFFEE700F0B7F820463D
:103C50000021FFF7FDF800F03BFE002818BF10BD63
:103C60004EF60450CEF200004FF080510160BFF3D9
:103C70004F8FBFF36F8F10BD44F66C51C2F200013D
:103C80000968016044F60461C2F2000109684160FC
:103C90007047000044F61060C2F20000012101608C
:103CA0007047000010B568B10C4640F2B851C2F23E
:103CB000000109681831FFF77BFE20460121FFF75C
:103CC000C7F810BD4FF0500080F31188BFF36F8F1D
:103CD000BFF34F8FFEE70000B0B590B10D4640F244
:103CE000B851C2F20001096814461831FFF77EFE90
:103CF000002C18BF4FF0FF3528462146FFF7A8F8E3
:103D0000B0BD4FF0500080F31188BFF36F8FBFF349
:103D10004F8F00BFFEE7000010B586B0002405A855
:103D200004A903AACDE90444FFF716FEDDE9032048
:103D300005990023CDE9010143F2BD10C0F6000052
:103D40001CA1009400F032FC44F66051C2F2000164
:103D5000086010B100F046FE0446601C20D0012C23
:103D60001CD14FF0500080F31188BFF36F8FBFF369
:103D70004F8F44F66850C2F200004FF0FF310160EF
:103D800044F6D050C2F200000121016044F6046004
:103D9000C2F200000021016000F066F806B010BD1C
:103DA0004FF0500080F31188BFF36F8FBFF34F8F38
:103DB000FEE700BF49444C450000000044F2446067
:103DC000C2F20000016801310160704744F24460B2
:103DD000C2F20000006830B144F61060C2F2000088
:103DE00001210160704744F61060C2F2000000211A
:103DF00044F24C6C0160C2F2000CDCF8001040F29E
:103E0000D05201EB8103C2F2000252F8230048B9FC
:103E100002EB8300A0F11403D9B153F8140901395E
:103E20000028F9D001EB810002EB800252F8040F68
:103E30004368101D8342136001D1586810601068F8
:103E400040F2B852C068C2F200021060CCF8001014
:103E500070474FF0500080F31188BFF36F8FBFF3AE
:103E60004F8F00BFFEE7000080B582B04EF20040E9
:103E7000CEF200004CF27021C4F20F11D0F80029EC
:103E80004B1C9A4209D14FF0500080F31188BFF3C8
:103E90006F8FBFF34F8F00BFFEE7D0F800298A4233
:103EA00009D14FF0500080F31188BFF36F8FBFF33B
:103EB0004F8F00BFFEE7017844F230620191FF218D
:103EC00001700178C2F200028DF803109DF8031012
:103ED00001F05001117044F23461C2F20001072276
:103EE0000A609DF90320B2F1FF3F0CDC0A6800BFB5
:103EF0009DF80330013A5B008DF803309DF90330E3
:103F0000002BF5D40A600A68032A2DD14FF4E06330
:103F100003EA02220A6001990170D0F8201941F4E5
:103F20007001C0F82019D0F8201941F07041C0F894
:103F30002019FFF7F5FD40F20C00C2F2000000214D
:103F40000160FFF761FD4EF63470CEF200000168AB
:103F500041F040410160FFF743FAFFF737FFFFF7F9
:103F6000CFFB002002B080BD4FF0500080F31188DD
:103F7000BFF36F8FBFF34F8FFEE7000080B54FF0A8
:103F8000500080F31188BFF36F8FBFF34F8F00F0A5
:103F900063FB30B14EF60450CEF200004FF080517A
:103FA0000160002080F3118880BD0000B0B582B0B0
:103FB00068B11D46ABB1F1B9EAB14FF0500080F3E2
:103FC0001188BFF36F8FBFF34F8F00BFFEE74FF035
:103FD000500080F31188BFF36F8FBFF34F8F00BF86
:103FE000FEE74FF0500080F31188BFF36F8FBFF3EF
:103FF0004F8F00BFFEE751B14AB94FF0500080F338
:104000001188BFF36F8FBFF34F8F00BFFEE75023C0
:104010000193019B502B0AD1069B019C012485F83A
:1040200046400095FFF7E0F8284602B0B0BD4FF0DB
:10403000500080F31188BFF36F8FBFF34F8F00BF25
:10404000FEE7000070B5F8B104460E46FFF7E6FC47
:104050002068D4E90F12002502FB0103013901FB9E
:104060000201A563C4E90103FF20E16084F8440074
:1040700084F8450004F110007EB1FFF789FC04F1DB
:104080002400FFF785FC18E04FF0500080F3118802
:10409000BFF36F8FBFF34F8FFEE7016869B100F088
:1040A000CFFB50B14EF60450CEF200004FF08051DD
:1040B0000160BFF34F8FBFF36F8FFFF7D3FC012079
:1040C00070BD00002DE9F04F83B00292B8B11D46DB
:1040D0000E460446E9B1022D03D1E06B012840F001
:1040E0009A8000F09FFA00BB0298F0B14FF05000A8
:1040F00080F31188BFF36F8FBFF34F8FFEE74FF050
:10410000500080F31188BFF36F8FBFF34F8F00BF54
:10411000FEE7206C0028DED04FF0500080F31188BD
:10412000BFF36F8FBFF34F8FFEE7FFF777FCA06BF6
:10413000022D58D0E16B884255D304F110080120BC
:104140006F464FF0000B0DF108094FF0805A00BF89
:104150000299002900F07B80C00702D03846FFF7A3
:104160008BFDFFF77FFCFFF729FEFFF757FC94F864
:104170004400FF2808BF84F844B094F84500FF28A5
:1041800008BF84F845B0FFF76DFC3846494600F09B
:1041900095F900285ED12046FFF714F9A0B10299E5
:1041A0004046FFF77FFD2046FFF7D0FA00F090FB76
:1041B00078B94EF60450CEF20000C0F800A0BFF36C
:1041C0004F8FBFF36F8F04E02046FFF7BFFA00F078
:1041D0007FFBFFF723FCA06B022D04D0E16B88422C
:1041E0004FF00000B4D2204631462A46FEF740FF89
:1041F00054F8241FC9B1204600F022FB08B34EF644
:104200000450CEF200004FF080510160BFF34F8F99
:10421000BFF36F8F15E04FF0500080F31188BFF3AC
:104220006F8FBFF34F8F00BFFEE750B14EF60450C3
:10423000CEF200004FF080510160BFF34F8FBFF30B
:104240006F8FFFF70FFC012003B0BDE8F08FFFF781
:1042500009FC04E02046FFF779FA00F039FB002062
:1042600003B0BDE8F08F00002DE9F04381B0E8B164
:104270001E46914605460F4609B3022E02D1E86B51
:10428000012837D1FFF766FCEFF311884FF050009B
:1042900080F31188BFF36F8FBFF34F8FA86B022E8F
:1042A00019D0E96B884216D300203FE04FF0500050
:1042B00080F31188BFF36F8FBFF34F8FFEE7286C39
:1042C0000028DAD04FF0500080F31188BFF36F8FD1
:1042D000BFF34F8FFEE795F84540A86B2846394657
:1042E0003246FEF7C5FEFF2C0DD0601C85F8450058
:1042F00001201BE04FF0500080F31188BFF36F8F57
:10430000BFF34F8FFEE755F8240F70B1284600F039
:1043100097FA0146B9F1000F4FF0010006D00029CD
:104320001CBF0120C9F8000000E0012088F31188BB
:1043300001B0BDE8F08300002DE9F04F85B0049294
:1043400098B10C460546002900F0A58000F06AF9F6
:10435000A8B9049898B14FF0500080F31188BFF3CA
:104360006F8FBFF34F8F00BFFEE74FF0500080F319
:104370001188BFF36F8FBFF34F8F00BFFEE705F1CA
:10438000240005F11009019002AF0DF1100A4FF061
:1043900000080AE02846FFF7D9F900F099FA284604
:1043A000FFF704F8002840F08480FFF737FBD5F8CA
:1043B00038B0BBF1000F1DD028462146FEF744FE61
:1043C000ABF10100A863286970B1484600F038FAE3
:1043D00050B14EF60450CEF200004FF08051016013
:1043E000BFF34F8FBFF36F8FFFF73CFB0020012619
:1043F000A0B95FE0049850B1B8F1000F02D138467F
:10440000FFF73AFC4FF00108012038B952E0FFF7FE
:1044100029FB0026002000284CD000BFFFF722FB1C
:10442000FFF7CCFCFFF7FAFA95F84400FF2804BF29
:10443000002085F8440095F84500FF2804BF0020BF
:1044400085F84500FFF70EFB3846514600F036F878
:1044500000289FD12846FEF7A9FFB0B10499019822
:10446000FFF720FC2846FFF771F900F031FA002829
:104470009BD14EF60450CEF200004FF08051016007
:10448000BFF34F8FBFF36F8F8FE72846FFF75EF9BB
:1044900000F01EFA89E7286C00283FF457AF4FF070
:1044A000500080F31188BFF36F8FBFF34F8F00BFB1
:1044B000FEE70026304605B0BDE8F08FB0B5D0B1BC
:1044C0000D4611B30446FFF7A9FA44F60460C2F2A0
:1044D000000001682868421C21D044F66C536268D1
:1044E000C2F20003D3F800C091421AD323689C455E
:1044F00017D0012422E04FF0500080F31188BFF361
:104500006F8FBFF34F8F00BFFEE74FF0500080F377
:104510001188BFF36F8FBFF34F8F00BFFEE70024FA
:104520000CE0891A884206D9401A28602046FFF715
:10453000A3FB002402E0002001242860FFF792FA88
:104540002046B0BD2DE9F04383B007469000984661
:1045500015468946FFF734F978B106465C20FFF727
:104560002FF938B10446066354B94FF0FF3003B059
:10457000BDE8F0833046FFF78DFA0024002CF4D01C
:10458000DDE90A10002284F85920CDE900103846F0
:1045900049462A4643460294FEF736FE2046FEF779
:1045A00097FC012003B0BDE8F083000070B586B031
:1045B0000B9CCCB10C9E06B35C250495049D5C2D30
:1045C00025D1049DDDF828C0022586F8595005AD97
:1045D0003463CDE900C50296FEF716FE3046FEF7BD
:1045E00077FC059806B070BD4FF0500080F311883D
:1045F000BFF36F8FBFF34F8FFEE74FF0500080F394
:104600001188BFF36F8FBFF34F8F00BFFEE74FF0EE
:10461000500080F31188BFF36F8FBFF34F8F00BF3F
:10462000FEE7000044F6D050C2F200000068002807
:1046300004BF0120704744F24460C2F200000068E9
:10464000B0FA80F0400940007047000044F6046072
:10465000C2F20000006870472DE9F04F81B044F2CB
:104660004460C2F20000006840B144F67850C2F2E3
:104670000000016800240131016092E044F604600A
:10468000C2F2000001684E1C066021D340F2C05007
:10469000C2F200000168096849B14FF0500080F390
:1046A0001188BFF36F8FBFF34F8F00BFFEE740F25B
:1046B000C852C2F2000201681368036044F66C50ED
:1046C0001160C2F20000016801310160FEF7A6FF2F
:1046D00044F66851C2F20001086840F2B85A40F24C
:1046E000D0588642C2F2000AC2F2000801D2002469
:1046F00045E040F2C057C2F2000738680024006865
:1047000098B344F24C6BC2F2000B19E0D9F82C00BC
:10471000DBF80010884288BFCBF8000000EB800077
:1047200008EB80002946FFF761F9D9F82C00DAF888
:104730000010C96A3A68884228BF01241068B8B1DD
:104740003868C068D0F80C904D4655F8040F864282
:1047500010D32846FFF7EEF8D9F828000028D5D066
:1047600009F11800FFF7E6F8D0E74FF0FF3005E059
:104770004FF0FF3044F66851C2F200010860DAF8E9
:104780000000C06A00EB800058F82000012844F6C1
:104790001060C2F2000088BF01240068002818BF22
:1047A0000124204601B0BDE8F08F0000B0B580B113
:1047B000044640F2B850C2F200000068A0420AD09D
:1047C0004FF0500080F31188BFF36F8FBFF34F8F0E
:1047D000FEE70020B0BD206D38B3013820654FF0F2
:1047E000000018BFB0BDE16AE26C91421CD0251DEB
:1047F0002846FFF79FF8E06CC0F13801A16144F250
:104800004C61E062C2F200010A68904288BF086011
:1048100040F2D05100EB8000C2F2000101EB8000B9
:104820002946FFF7E3F80120B0BD4FF0500080F3B8
:104830001188BFF36F8FBFF34F8F00BFFEE70000FB
:10484000B0B5C068C5687DB105F118042046FFF712
:1048500071F844F24460C2F20000006868B144F6A6
:104860007C50C2F200001DE04FF0500080F3118830
:10487000BFF36F8FBFF34F8FFEE72C1D2046FFF76E
:1048800059F844F24C61C2F20001E86A0A689042A9
:1048900088BF086040F2D05100EB8000C2F20001F6
:1048A00001EB80002146FFF7A1F840F2B851C2F2B7
:1048B0000001E86A0968C96A884291BF002044F68D
:1048C0001061C2F20001012088BF0860B0BD000085
:1048D0002DE9F04F81B044F24464C2F20004206834
:1048E00068B1FFF79BF8206801382060206880B12C
:1048F0000024FFF7B7F8204601B0BDE8F08F4FF075
:10490000500080F31188BFF36F8FBFF34F8F00BF4C
:10491000FEE744F23C60C2F20000006800285DD06F
:1049200044F67C56C2F20006306844F61068C2F2C3
:10493000000890B344F24C6740F2D05940F2B85BA3
:10494000C2F20007C2F20009C2F2000B4FF0010AE6
:10495000F068C56805F11800FEF7ECFF2C1D204635
:10496000FEF7E8FFE86A3968884288BF386000EBE4
:10497000800009EB80002146FFF738F8E86ADBF891
:104980000010C96A884228BFC8F800A03068002813
:10499000DED1002D18BFFEF741FE44F67854C2F276
:1049A0000004256855B10126FFF756FE002818BF00
:1049B000C8F80060013DF7D100202060D8F8000061
:1049C00070B14EF60450CEF200004FF080510160FD
:1049D000BFF34F8F0124BFF36F8F8AE7002488E76E
:1049E000002486E780B586B0FEF7C8FA44F6086072
:1049F000C2F20000006808B30020CDE9040005A859
:104A000004A903AAFEF7B6FFDDE903200221DDF8C1
:104A100014C0CDE9001043F23570C0F600000CA1BF
:104A20000023CDF808C0FFF7C1FD44F60C61C2F2C7
:104A30000001086010B1012006B080BD4FF05000A9
:104A400080F31188BFF36F8FBFF34F8FFEE700BF76
:104A5000546D72205376630010B584B0A8B144F64B
:104A60000864C2F2000484462068C0B10529CDE97B
:104A70000012CDF808C015DCFFF7D4FD0146206810
:104A8000022916D1069A694615E04FF0500080F3CE
:104A90001188BFF36F8FBFF34F8F00BFFEE7002079
:104AA00004B010BD69461A460023FFF7DDFB04B0D1
:104AB00010BD694600220023FFF704FB04B010BDBF
:104AC000F1EE100A4FF6FF71C0F2C03120EA01008A
:104AD00040F04070E1EE100A704700000000000056
:104AE000000001020304060708090000000001029B
:104AF00003040000184B0008000000000000000044
:104B0000000000000000000000020000180000008B
:104B1000000000000000000064656661756C74545C
:104B200061736B00484B000800000020100000007B
:104B3000C4010008584B0008100000200854000071
:104B4000E0010008000000000024F4000100000063
:084B500010000000AAAAAAAAA5
:040000050800018965
:00000001FF
